:100000000C9434000C9451000C9451000C94510049
:100010000C9451000C9451000C9451000C9451001C
:100020000C9451000C9451000C9451000C9451000C
:100030000C9451000C9451000C9451000C945100FC
:100040000C9451000C9451000C94B4000C94F400E6
:100050000C9451000C9451000C9451000C945100DC
:100060000C9451000C94510011241FBECFEFD8E026
:10007000DEBFCDBF11E0A0E0B1E0E6EDF9E002C0E7
:1000800005900D92A432B107D9F713E0A4E2B1E0D4
:1000900001C01D92A237B107E1F70E9453010C94F1
:1000A000E9040C9400000E94430108951092250376
:1000B00010922403109227031092260310926903D2
:1000C0001092680310926B0310926A031092C5009D
:1000D00087E68093C40086E08093C20088E1809325
:1000E000C100789408951F93182F8A3019F48DE079
:1000F0000E9473002091260330912703C9010196C5
:1001000060E071E00E94C5014091240350912503F5
:100110008417950781F0F901EE0FFF1FEC5DFE4F8C
:100120001083118290932703809326038091C1004E
:1001300080628093C10080E090E01F9108958091DB
:10014000680390916903019660E270E00E94C50126
:100150009093690380936803FC01EE0FFF1FE85D35
:10016000FC4F8081918108951F920F920FB60F92DC
:1001700011242F933F934F935F936F937F938F93AC
:100180009F93AF93BF93EF93FF9320916A033091B6
:100190006B03C901019660E270E00E94C5014091C5
:1001A0006803509169038417950769F04091C60070
:1001B000F901EE0FFF1FE85DFC4F40831182909321
:1001C0006B0380936A03FF91EF91BF91AF919F9171
:1001D0008F917F916F915F914F913F912F910F90F0
:1001E0000FBE0F901F9018951F920F920FB60F928F
:1001F00011242F933F935F936F937F938F939F93DC
:10020000AF93BF93EF93FF938091240390912503C5
:10021000019660E071E00E94C501209126033091B3
:1002200027038217930769F0FC01EE0FFF1FEC5DB7
:10023000FE4F20812093C6009093250380932403D2
:1002400005C08091C1008F7D8093C100FF91EF9127
:10025000BF91AF919F918F917F916F915F913F91EE
:100260002F910F900FBE0F901F901895259A239AEB
:10027000229A8CB58F7D8CBD8CB580618CBD8CB580
:1002800080648CBD0895CF93DF930F92CDB7DEB716
:10029000898389818EBD0DB407FEFDCF8EB50F9089
:1002A000DF91CF910895CF93DF93CDB7DEB76197FC
:1002B0000FB6F894DEBF0FBECDBF0E9456000E945D
:1002C000360186E191E090936F0380936E0388E09E
:1002D00091E090936D0380936C038AEA0E9453002F
:1002E00080EF0E9453002A982A9A80E593EC20E937
:1002F00031E0F9013197F1F70197D9F700E010E00B
:100300007E010894E11CF11C80E0C82E81E0D82E0B
:1003100090E9A92E91E0B92EC801B70142E050E062
:100320000E94EC0100D000D000D0EDB7FEB73196AE
:10033000ADB7BEB71296DC92CE921197F382E282ED
:10034000158304830E940D028DB79EB706960FB6E3
:10035000F8949EBF0FBE8DBF812F0E945300802F47
:100360000E9453002A982A9A24EF31E0C501019790
:10037000F1F721503040D1F70F5F1F4F9FEF0F3F34
:10038000190751F600E010E0C7CF97FB092E0726AA
:100390000AD077FD04D00CD006D000201AF4709556
:1003A00061957F4F0895F6F7909581959F4F089539
:1003B000AA1BBB1B51E107C0AA1FBB1FA617B7078B
:1003C00010F0A61BB70B881F991F5A95A9F78095A7
:1003D0009095BC01CD010895FB019F01E894423046
:1003E000C4F04532B4F44A3029F497FB1EF49095DA
:1003F00081959F4F642F77270E94D801805D8A33B3
:100400000CF0895D8193CB010097A1F716F45DE2B2
:1004100051931082C9010C941804A0E0B0E0E3E10C
:10042000F2E00C94C204FE013596619171918091C5
:100430006E0390916F03AF010E9422022096E2E0CA
:100440000C94DE04ADE0B0E0E8E2F2E00C94B2041B
:100450003C017D876C875A01FC01178216828381DB
:1004600081FFCAC13FE3C32E2E010894411C511CD9
:10047000F3019381EC85FD8593FD859193FF819137
:10048000FD87EC87882309F4B3C1853241F493FDDD
:10049000859193FF8191FD87EC87853229F490E067
:1004A000B3010E942804E4CFEE24DD2410E01032D2
:1004B000B0F48B3269F08C3228F4803251F0833200
:1004C00071F40BC08D3239F0803349F411602CC0C7
:1004D0001260146029C0186027C0106125C017FD84
:1004E0002EC0282F20532A3098F416FF08C08E2DD6
:1004F000880FE82EEE0CEE0CE80EE20E15C08D2DE6
:10050000880FD82EDD0CDD0CD80ED20E10620CC078
:100510008E3221F416FD6CC1106406C08C3611F4C5
:10052000106802C0883659F4EC85FD8593FD8591ED
:1005300093FF8191FD87EC87882309F0B8CF982F2E
:100540009554933018F09052933030F424E030E01A
:10055000A20EB31EC9820FC0833631F0833781F0FB
:10056000833509F05AC022C0F5018081898322E0D9
:1005700030E0A20EB31E21E0E22EF12C420114C0A5
:1005800092E0292E312C2A0C3B1CF50180809180B1
:1005900016FF03C06E2D70E002C06FEF7FEFC40145
:1005A0000E940D047C0151011F7715C082E0282EA6
:1005B000312C2A0C3B1CF5018080918016FF03C072
:1005C0006E2D70E002C06FEF7FEFC4010E94020445
:1005D0007C011068510113FD1CC006C080E290E050
:1005E000B3010E942804DA948D2D90E0E816F906F4
:1005F000A8F30FC0F40117FD859117FF81914F01FA
:1006000090E0B3010E942804D110DA940894E10824
:10061000F108E114F10471F7E8C0843611F089366D
:1006200059F5F50117FF07C080819181A281B3813F
:1006300024E030E009C060817181CB01AA2797FDD9
:10064000A095BA2F22E030E0A20EB31E012F0F7644
:10065000B7FF08C0B095A095909581959F4FAF4F7B
:10066000BF4F0068BC01CD01A2012AE030E00E942A
:100670005404F82EF4183FC0853721F41F7E2AE079
:1006800030E020C0197F8F36A9F0803720F48835FC
:1006900009F0AEC00BC0803721F0883709F0A8C040
:1006A00001C0106114FF09C0146007C014FF08C026
:1006B000166006C028E030E005C020E130E002C04E
:1006C00020E132E0F50117FF07C06081718182816E
:1006D000938144E050E006C06081718180E090E049
:1006E00042E050E0A40EB51EA2010E945404F82E70
:1006F000F418012F0F7706FF09C00E7FFE1430F4A7
:1007000004FF06C002FD04C00F7E02C01F2D01C001
:100710001E2D802F90E004FF0CC0FE01EF0DF11D97
:100720002081203311F4097E09C002FF06C01E5F3C
:1007300005C086789070009709F01F5F802E99247D
:1007400003FD12C000FF0DC0EF2C1D1550F4ED0C81
:10075000E11A1D2D06C080E290E0B3010E9428043A
:100760001F5F1D15C0F304C01D1510F4D11A01C080
:10077000DD2484FE0FC080E390E0B3010E942804D2
:1007800082FE1FC081FE03C088E590E010C088E7AC
:1007900090E00DC0C40186789070009791F081FCC4
:1007A00002C080E201C08BE207FD8DE290E0B30160
:1007B0000E94280406C080E390E0B3010E94280450
:1007C000EA94FE14C0F3FA94F201EF0DF11D80815A
:1007D00090E0B3010E942804FF20A9F706C080E240
:1007E00090E0B3010E942804DA94DD20C1F740CEE6
:1007F000F3018681978102C08FEF9FEF2D96E2E192
:100800000C94CE04FC010590615070400110D8F7A3
:10081000809590958E0F9F1F0895FC016150704048
:1008200001900110D8F7809590958E0F9F1F089525
:10083000DC01FC01672F71917723E1F7329704C047
:100840007C916D9370836291AE17BF07C8F30895D2
:100850000F931F93CF93DF938C01EB018B8181FF6B
:100860001BC082FF0DC02E813F818C819D81281786
:10087000390764F4E881F9810193F983E88306C0BC
:10088000E885F985802F0995009731F48E819F8145
:1008900001969F838E8302C00FEF1FEFC801DF9187
:1008A000CF911F910F910895FA01AA27283051F195
:1008B000203181F1E8946F936E7F6E5F7F4F8F4F91
:1008C0009F4FAF4FB1E03ED0B4E03CD0670F781FF0
:1008D000891F9A1FA11D680F791F8A1F911DA11DD5
:1008E0006A0F711D811D911DA11D20D009F468940E
:1008F0003F912AE0269F11243019305D3193DEF6B6
:10090000CF010895462F4770405D4193B3E00FD06B
:10091000C9F7F6CF462F4F70405D4A3318F0495D56
:1009200031FD4052419302D0A9F7EACFB4E0A69539
:100930009795879577956795BA95C9F7009761055B
:10094000710508959B01AC010A2E069457954795B1
:1009500037952795BA95C9F7620F731F841F951FA6
:10096000A01D08952F923F924F925F926F927F92B7
:100970008F929F92AF92BF92CF92DF92EF92FF92AF
:100980000F931F93CF93DF93CDB7DEB7CA1BDB0B5B
:100990000FB6F894DEBF0FBECDBF09942A88398800
:1009A00048885F846E847D848C849B84AA84B98407
:1009B000C884DF80EE80FD800C811B81AA81B98113
:1009C000CE0FD11D0FB6F894DEBF0FBECDBFED0127
:0609D0000895F894FFCF2A
:1009D6002573202564200A000000000100000000A5
:1009E60000009F00000000000002000000007300ED
:0409F60000000000FD
:00000001FF
